:1000000000308A001C2900000A108A100A11820799
:1000100028340C34013406340A108A100A1182077D
:100020004234613474346534723469346534203454
:100030006A34653420346E34613462346934743423
:10004000613420346E34613400340A108A100A118D
:100050008207413454342B344334423443340D3416
:1000600000340A108A100A118207253463342534BB
:1000700063342034703472346F34633465346E34D6
:10008000743400343730840083130008031959286E
:100090000130F800BF30F7006400F70B4C28F80B74
:1000A0004A284A30F700F70B532800006400800B01
:1000B000482800340708F039BE003D080F393E04D7
:1000C000870006148316061064002030F700F70B33
:1000D00067286A28831206108316061083120034DC
:1000E000BB08031D75288610762886148316861093
:1000F0008312BC0E3C08BD005A20BC0E3C08BD005B
:100100005A2064004230F700F70B84280034143082
:10011000B7004220F03083168705831286108316BD
:10012000861083120610831606108312B501350857
:10013000023C031CA3280230B70042200330BD005C
:100140005A20B50A972864000C30F700F70BA62850
:10015000A9280230BD005A2064000C30F700F70BCC
:10016000AF28B228B5013508023C031CC328350866
:100170000420B600BB013608BC0070200230B70076
:100180004220B50AB3286D2901303802FC3E03181D
:10019000D628043EE128B901D6284030B900D62837
:1001A0001430B900D6285430B900D62801303702AF
:1001B000B90739088038BA00BB013A08BC00702082
:1001C00000340A108A100A118207CB28CD28D028C3
:1001D000D32836080C3A0319F728063A0319FF28E2
:1001E000073A03190529053A03190A290F29BB0102
:1001F0000130BC0070200230B70042201B290130C2
:10020000B7000230B800C4201B290130B700B80085
:10021000C4201B29BB011030BC0070201B293608EC
:100220001F3C031C15290730B6050130BB003608FA
:10023000BC0070201B290034840183131F30830508
:100240000C3083169900A6309800903083129800E5
:1002500083161F149F141F159F1107309C00FF3039
:100260008312B40083161F149F141F159F1183124D
:100270001F108316091283129412B41234088316C5
:100280008700831234163408831687008312B41152
:1002900034088316870001308312940000308316DF
:1002A00094000108C739083881008312900100309A
:1002B000F800920000308316920007309C00050879
:1002C00064000230F700F70B632966291C088312CB
:1002D0000D1383169D01831287289630B7004220A4
:1002E000B50135080C20B50AF700B600E920143036
:1002F0003502031D7129B50135082520B50AF7001F
:1003000077080C1E8129990007303502031D7C29CE
:100310002030840083138403840A8C1E8D291A08DC
:1003200080000D300002031D8C2980018C1E96294F
:100330001A082030840083138403840A8C1E9E29AB
:100340001A0880000D300002031D9D29800106302F
:10035000B7000230B800C4202908B600E9202A08F6
:10036000B600E9200430B50035083120B50AF700A1
:10037000B600E9200C303502031DB4290A30B5005F
:0E038000FA30B7004220B50BC0297B2963007C
:02400E00393F38
:00000001FF
